:020000040800F2
:10000000004000205D290008BD170008BF17000848
:10001000C1170008C3170008C5170008000000003A
:10002000000000000000000000000000C7170008EA
:10003000C917000800000000CB170008CD17000802
:10004000AD290008AD290008AD290008AD29000838
:10005000AD290008AD290008AD290008AD29000828
:10006000AD290008AD290008AD290008AD29000818
:10007000AD290008AD290008AD290008AD29000808
:10008000AD290008AD290008AD290008AD290008F8
:10009000AD290008AD290008AD290008AD290008E8
:1000A000AD290008AD290008AD290008AD290008D8
:1000B000AD2900080000000000000000AD29000884
:1000C000AD290008AD290008AD2900080000000096
:1000D000AD290008AD290008AD290008AD290008A8
:1000E000AD290008AD290008AD2900080000000076
:1000F0000000000000000000000000000000000000
:10010000000000000000000000000000AD29000811
:100110000000000000000000AD2900080000000001
:1001200000000000000000000000000000000000CF
:1001300000000000000000000000000000000000BF
:10014000AD290008AD2900080000000000000000F3
:10015000000000000000000000000000000000009F
:10016000AD290008AD290008AD290008AD29000817
:10017000AD290008000000000000000000000000A1
:0801800000000000AD29000899
:1001880070B54FF0FF0C4CF4E06C1CEA11541DBF25
:100198001CEA135594EA0C0F95EA0C0F00F0DEF8F0
:1001A8002C4481EA030621EA4C5123EA4C5350EAD5
:1001B800013518BF52EA033541F4801143F4801326
:1001C80038D0A0FB02CE4FF00005E1FB02E506F0B7
:1001D8000042E0FB03E54FF00006E1FB03569CF00C
:1001E800000F18BF4EF0010EA4F1FF04B6F5007F12
:1001F80064F5407404D25FEA4E0E6D4146EB060684
:1002080042EAC62141EA55514FEAC52040EA5E500C
:100218004FEACE2EB4F1FD0C88BFBCF5E06F1ED8B6
:10022800BEF1004F08BF5FEA500E50F1000041EBED
:10023800045170BD06F0004646EA010140EA02009A
:1002480081EA0301B4EB5C04C2BFD4EB0C0541EABC
:10025800045170BD41F480114FF0000E013C00F3D1
:10026800AB8014F1360FDEBF002001F0004170BDF5
:10027800C4F10004203C35DA0C341BDC04F114040E
:10028800C4F1200500FA05F320FA04F001FA05F29A
:1002980040EA020001F0004221F0004110EBD37067
:1002A80021FA04F642EB06015EEA430E08BF20EA93
:1002B800D37070BDC4F10C04C4F1200500FA04F336
:1002C80020FA05F001FA04F240EA020001F00041C8
:1002D80010EBD37041F100015EEA430E08BF20EA3B
:1002E800D37070BDC4F1200500FA05F24EEA020E83
:1002F80020FA04F301FA05F243EA020321FA04F0B2
:1003080001F0004121FA04F220EA020000EBD37068
:100318005EEA430E08BF20EAD37070BD94F0000F68
:100328000FD101F00046400041EB010111F4801F9C
:1003380008BF013CF7D041EA060195F0000F18BF4D
:10034800704703F00046520043EB030313F4801F89
:1003580008BF013DF7D043EA0603704794EA0C0F43
:100368000CEA135518BF95EA0C0F0CD050EA410659
:1003780018BF52EA4306D1D181EA030101F00041D6
:100388004FF0000070BD50EA410606BF10461946FE
:1003980052EA430619D094EA0C0F02D150EA01360A
:1003A80013D195EA0C0F05D152EA03361CBF10464B
:1003B80019460AD181EA030101F0004141F0FE41EA
:1003C80041F470014FF0000070BD41F0FE4141F46E
:1003D800780170BD81F0004102E000BF83F0004366
:1003E80030B54FEA41044FEA430594EA050F08BFC8
:1003F80090EA020F1FBF54EA000C55EA020C7FEA8C
:10040800645C7FEA655C00F0E2804FEA5454D4EB08
:100418005555B8BF6D420CDD2C4480EA020281EAD2
:10042800030382EA000083EA010180EA020281EA0A
:100438000303362D88BF30BD11F0004F4FEA01315C
:100448004FF4801C4CEA113102D0404261EB41016B
:1004580013F0004F4FEA03334CEA133302D05242F1
:1004680063EB430394EA050F00F0A780A4F10104AD
:10047800D5F1200E0DDB02FA0EFC22FA05F28018E7
:1004880041F1000103FA0EF2801843FA05F35941CD
:100498000EE0A5F120050EF1200E012A03FA0EFC4C
:1004A80028BF4CF0020C43FA05F3C01851EBE37176
:1004B80001F0004507D54FF0000EDCF1000C7EEB93
:1004C80000006EEB0101B1F5801F1BD3B1F5001FD1
:1004D8000CD349085FEA30004FEA3C0C04F10104F0
:1004E8004FEA445212F5800F80F09A80BCF1004F19
:1004F80008BF5FEA500C50F1000041EB045141EA9B
:10050800050130BD5FEA4C0C404141EB0101013C63
:1005180028BFB1F5801FE9D291F0000F04BF014652
:100528000020B1FA81F308BF2033A3F10B03B3F124
:1005380020020CDA0C3208DD02F1140CC2F10C02B4
:1005480001FA0CF021FA02F10CE002F11402D8BF12
:10055800C2F1200C01FA02F120FA0CFCDCBF41EADE
:100568000C019040E41AA2BF01EB0451294330BDAD
:100578006FEA04041F3C1CDA0C340EDC04F114048A
:10058800C4F1200220FA04F001FA02F340EA030061
:1005980021FA04F345EA030130BDC4F10C04C4F1A7
:1005A800200220FA02F001FA04F340EA0300294687
:1005B80030BD21FA04F0294630BD94F0000F83F4D1
:1005C800801306BF81F480110134013D4EE77FEAB4
:1005D800645C18BF7FEA655C29D094EA050F08BF00
:1005E80090EA020F05D054EA000C04BF19461046E1
:1005F80030BD91EA030F1EBF0021002030BD5FEA25
:10060800545C05D14000494128BF41F0004130BD4C
:1006180014F580043CBF01F5801130BD01F00045A0
:1006280045F0FE4141F470014FF0000030BD7FEA13
:10063800645C1ABF194610467FEA655C1CBF0B460E
:10064800024650EA013406BF52EA033591EA030F25
:1006580041F4002130BD00BF90F0000F04BF00211D
:10066800704730B54FF4806404F132044FF0000550
:100678004FF0000150E700BF90F0000F04BF0021C9
:10068800704730B54FF4806404F1320410F000452F
:1006980048BF40424FF000013EE700BF42004FEA2A
:1006A800E2014FEA31014FEA02701FBF12F07F43A7
:1006B80093F07F4F81F06051704732F07F4208BF5E
:1006C800704793F07F4F04BF41F40021704730B565
:1006D8004FF4607401F0004521F000411CE700BFB1
:1006E80050EA010208BF704730B54FF000050AE034
:1006F80050EA010208BF704730B511F0004502D535
:10070800404261EB41014FF4806404F132045FEA36
:10071800915C3FF4D8AE4FF003025FEADC0C18BFDF
:1007280003325FEADC0C18BF033202EBDC02C2F1D1
:10073800200300FA03FC20FA02F001FA03FE40EA63
:100748000E0021FA02F11444BDE600BF4FEA41024F
:1007580012F5001215D211D56FF47873B3EB62520B
:1007680012D94FEAC12343F0004343EA505311F032
:10077800004F23FA02F018BF404270474FF00000C4
:10078800704750EA013005D111F0004008BF6FF002
:10079800004070474FF00000704700BF4A0011D278
:1007A80012F5001211D20DD56FF47873B3EB6252C3
:1007B8000ED44FEAC12343F0004343EA505323FACF
:1007C80002F070474FF00000704750EA013002D144
:1007D8004FF0FF3070474FF00000704710B5054CE0
:1007E800237833B9044B13B10448AFF300800123D5
:1007F800237010BD1000002000000000082A000827
:1008080008B5034B1BB103490348AFF3008008BD8B
:100818000000000014000020082A000800B583B07A
:1008280006226946022000F0F9FD03B05DF804FBDA
:1008380010B584B0044600230293ADF80C300622AC
:1008480002A9322000F0EAFD08B104B010BD9DF8FD
:1008580008309DF8092043EA0223A3869DF80A3050
:100868009DF80B2043EA0223E28E63F3CF02E2866F
:100878009DF80C30D90994F8382061F3000284F807
:100888003820C3F38011D2B261F3410284F83820D2
:10089800C3F34011D2B261F3820284F83820C3F363
:1008A8000011D2B261F3C30284F83820C3F3C00147
:1008B800D2B261F3041284F83820C3F38001D2B2B3
:1008C80061F3451284F83820C3F34001D2B261F3D2
:1008D800861284F83820D2B263F3C71284F838201D
:1008E8009DF80D30D90994F8392061F3000284F895
:1008F8003920C3F38011D2B261F3410284F8392060
:10090800C3F34011D2B261F3820284F83920C3F3F1
:100918000011D2B261F3C30284F83920C3F3C001D5
:10092800D2B261F3041284F83920C3F38001D2B241
:1009380061F3451284F83920C3F34001D2B261F360
:10094800861284F83920D2B263F3C71284F83920AA
:1009580040F21E7000F099FD00283FF476AF0622A1
:1009680002A9192000F05AFD00287FF46EAF9DF807
:1009780008009DF8093040EA032000B2FFF77CFE2A
:10098800A5A3D3E90023FFF7FBFBA5A3D3E9002325
:10099800FFF726FDFFF7DAFE20849DF80A009DF890
:1009A8000B3040EA032000B2FFF766FE9AA3D3E9B2
:1009B8000023FFF7E5FB9AA3D3E90023FFF710FD17
:1009C800FFF7C4FE60849DF80C009DF80D3040EAE6
:1009D800032000B2FFF750FE8FA3D3E90023FFF7EF
:1009E800CFFB8FA3D3E90023FFF7FAFCFFF7AEFE96
:1009F800A084062202A91A2000F010FD00287FF426
:100A080024AF9DF808009DF8093040EA032000B2A1
:100A1800FFF732FE80A3D3E90023FFF7B1FB80A3E1
:100A2800D3E90023FFF7DCFCFFF790FEE0849DF894
:100A38000A009DF80B3040EA032000B2FFF71CFEC5
:100A480075A3D3E90023FFF79BFB75A3D3E9002324
:100A5800FFF7C6FCFFF77AFE20859DF80C009DF88D
:100A68000D3040EA032000B2FFF706FE6AA3D3E97F
:100A78000023FFF785FB6AA3D3E90023FFF7B0FC47
:100A8800FFF764FE6085062202A91B2000F0C6FC61
:100A980000287FF4DAAE9DF808009DF8093040EA96
:100AA800032000B2FFF7E8FD5BA3D3E90023FFF7BB
:100AB80067FB5BA3D3E90023FFF792FCFFF746FE31
:100AC800A0859DF80A009DF80B3040EA032000B28B
:100AD800FFF7D2FD50A3D3E90023FFF751FB50A342
:100AE800D3E90023FFF77CFCFFF730FEE0859DF893
:100AF8000C009DF80D3040EA032000B2FFF7BCFD62
:100B080045A3D3E90023FFF73BFB45A3D3E9002323
:100B1800FFF766FCFFF71AFE2086062202A91F20AF
:100B280000F07CFC00287FF490AE9DF808009DF84A
:100B3800093040EA032000B2FFF79EFD36A3D3E94F
:100B48000023FFF71DFB36A3D3E90023FFF748FC7A
:100B5800FFF7FCFD608606226946302000F05EFC47
:100B680000287FF472AE9DF802309DF8032043EA16
:100B78000223638706226946312000F04FFC0028D3
:100B88007FF463AE9DF800009DF8013040EA032031
:100B980000B2FFF771FD20A3D3E90023FFF7F0FAB5
:100BA8001FA3D3E90023FFF71BFCFFF7F7FDE0873E
:100BB8009DF802009DF8033040EA032000B2FFF7D9
:100BC8005BFD15A3D3E90023FFF7DAFA14A3D3E9F1
:100BD8000023FFF705FCFFF7E1FDA0879DF804005F
:100BE8009DF8053040EA032000B2FFF745FD0AA34F
:100BF800D3E90023FFF7C4FA09A3D3E90023FFF7D9
:100C0800EFFBFFF7CBFDA4F84200002211464FF49A
:100C1800826000F0ABFB18E6333333333333C33F22
:100C2800000000000070974008B5002211462820F7
:100C380000F09CFB08BDB1F5805F30D230B583B0C1
:100C480005460C46B0F5805F02D3012003B030BDE5
:100C580006226946262000F0E1FB0028F6D18DF82F
:100C680000409DF8013003F0F0038DF80130C4F323
:100C7800032423438DF8013003F00F038DF801306E
:100C88002A01D2B213438DF80130C5F307158DF848
:100C9800025006226946242000F068FBD6E70120AE
:100CA8007047000000B583B0FFF7B8FD0022114679
:100CB800272000F0B3FB0A2000F009FCFFF7AEFD87
:100CC800FFF7B2FF40F2A11140F26540FFF7B3FF12
:100CD800154B93E803000090ADF80410062269460E
:100CE80040F2177000F042FB034618B1184603B0F3
:100CF8005DF804FB0622694640F2157000F036FBE9
:100D080003460028F2D1002211464FF4787000F013
:100D18002DFB03460028E9D1002211464FF48260DA
:100D280000F024FB0346E1E7202A000838B50D4609
:100D3800144600F0EBFA034B1D70034B1C70FFF7D1
:100D4800B1FF38BD2D0000202C00002010B582B066
:100D5800044606226946332000F060FB38BB9DF844
:100D680000E09DF801304EEA032E9DF802304EEA6D
:100D7800034E9DF803304EEA036E0022A265E26539
:100D880011E0E16D53002EFA03FC0CF0010C41EA6E
:100D98000C01E165A16D01332EFA03F303F00103A1
:100DA8001943A1650132034B1B789342E9D802B07D
:100DB80010BD00BF2D00002030B583B004460622C8
:100DC8006946042000F02AFB054610B1284603B006
:100DD80030BD9DF800009DF8013040EA032000B2C4
:100DE800FFF74AFCC2A3D3E90023FFF7C9F9C2A35E
:100DF800D3E90023FFF7F4FAFFF7A8FC20809DF859
:100E080002009DF8033040EA032000B2FFF734FCEB
:100E1800B7A3D3E90023FFF7B3F9B7A3D3E90023B6
:100E2800FFF7DEFAFFF792FC60809DF804009DF85A
:100E3800053040EA032000B2FFF71EFCACA3D3E95B
:100E48000023FFF79DF9ACA3D3E90023FFF7C8FA05
:100E5800FFF77CFCA08006226946104600F0DEFA07
:100E680005460028B2D19DF800009DF8013040EAFF
:100E7800032000B2FFF700FC9DA3D3E90023FFF78E
:100E88007FF99DA3D3E90023FFF7AAFAFFF75EFCD9
:100E9800E0809DF802009DF8033040EA032000B28C
:100EA800FFF7EAFB92A3D3E90023FFF769F992A3BE
:100EB800D3E90023FFF794FAFFF748FC20819DF857
:100EC80004009DF8053040EA032000B2FFF7D4FB88
:100ED80087A3D3E90023FFF753F987A3D3E90023B6
:100EE800FFF77EFAFFF732FC608106226946082088
:100EF80000F094FA054600287FF468AF9DF80000DA
:100F08009DF8013040EA032000B2FFF7B5FB78A353
:100F1800D3E90023FFF734F977A3D3E90023FFF7D8
:100F28005FFAFFF713FCA0819DF802009DF80330DB
:100F380040EA032000B2FFF79FFB6DA3D3E900232B
:100F4800FFF71EF96CA3D3E90023FFF749FAFFF76F
:100F5800FDFBE0819DF804009DF8053040EA032080
:100F680000B2FFF789FB62A3D3E90023FFF708F972
:100F780061A3D3E90023FFF733FAFFF7E7FB2082E9
:100F8800062269460A2000F049FA054600287FF43F
:100F98001DAF9DF800009DF8013040EA032000B223
:100FA800FFF76AFB52A3D3E90023FFF7E9F852A33E
:100FB800D3E90023FFF714FAFFF7C8FB60829DF816
:100FC80002009DF8033040EA032000B2FFF754FB0B
:100FD80047A3D3E90023FFF7D3F847A3D3E90023B6
:100FE800FFF7FEF9FFF7B2FBA0829DF804009DF819
:100FF800053040EA032000B2FFF73EFB3CA3D3E9EB
:101008000023FFF7BDF83CA3D3E90023FFF7E8F975
:10101800FFF79CFBE08206226946092000F0FEF9F2
:10102800054600287FF4D2AE9DF800009DF80130F7
:1010380040EA032000B2FFF71FFB2DA3D3E90023EA
:10104800FFF79EF82CA3D3E90023FFF7C9F9FFF7B0
:101058007DFB20839DF802009DF8033040EA0320C1
:1010680000B2FFF709FB22A3D3E90023FFF788F8B2
:1010780021A3D3E90023FFF7B3F9FFF767FB6083E8
:101088009DF804009DF8053040EA032000B2FFF700
:10109800F3FA17A3D3E90023FFF772F816A3D3E9ED
:1010A8000023FFF79DF9FFF751FBA083062269464D
:1010B8000B2000F0B3F9054600287FF487AE9DF8B1
:1010C80000009DF8013040EA032000B2FFF7D4FA8F
:1010D80007A3D3E90023FFF753F807A3D3E90023B5
:1010E800FFF77EF9FFF732FBE0836FE6AFF300808E
:1010F800333333333333C33F00000000007097406D
:1011080008B5FFF759FE08BD8000002303E0400042
:1011180080B20133DBB2072B07D810F4007FF6D07A
:10112800400080F08F0080B2F3E7704770B5C0F3DD
:10113800803282EAD1131946C0F380025A40C0F3C4
:10114800C00C83EA0C0CC0F3801E83EA0E0EC0F3B9
:10115800C0145C40C0F340255D40C0F340365E409B
:10116800400000F4005343EA863300F480563343CA
:101178001BB200F40066334343EA852300F400758C
:101188002B431BB243EA042343EACE1300F0400486
:1011980023431BB200F02004234343EA0C1343EA21
:1011A800C20300F0040213431BB200F00200034321
:1011B8009BB241EA030070BD02290FD80120704795
:1011C800715DA140C9B2FFF7B1FF0134072CF7DD0B
:1011D8000135BB1EAB4207DD0024F7E7F8B506462C
:1011E8000F4600251020F4E7C209F254013F4300DE
:1011F800F3550020F8BD10B504464FF0000C10233D
:1012080010E05B009BB20138C0B238B113F4007F24
:10121800F7D05B009BB283F08F03F4E70CF1010C6D
:101228005FFA8CFC8C4505DA12F80CE083EA8E0331
:101238000820EAE79CB1525C920002F47C725340A9
:10124800062203E05B009BB2013AD2B23AB113F432
:10125800007FF7D05B009BB283F08F03F4E7C3F302
:10126800090010BD022901D80120704770B582B06D
:1012780005460C468E1E024631460120FFF7BBFF8D
:10128800C0F30123AB55631EE8542A4621460120CA
:10129800FFF7B1FFC0B28DF80700002002B070BDA3
:1012A800F8B507460E46002510240BE0C4F3870066
:1012B8007B5D5840FFF728FF2402A4B2604084B247
:1012C80001352DB2B542F1DBC4F30900F8BD02299E
:1012D80006D908B5FFF7E4FF003818BF012008BD9C
:1012E800FF20704708B500224021024800F01EFC8C
:1012F80008BD00BF0004004808B50122402102488B
:1013080000F014FC08BD00BF0004004810B50446F6
:10131800FFF7E8FF012000F0ADFAFFF7EDFF024B01
:101328001C60002010BD00BF3000002090B585B0C3
:1013380002AF0B46CA1D02F4FC72ADEB020D6A4601
:10134800094C642142F8081B0146206801F08BF91A
:1013580000237B6023681B68DA687A609B687B607F
:101368007B680C37BD4690BD300000202DE9F04168
:1013780082B000AF82B30D461446E84602F10D0371
:1013880003F4FC73ADEB030D6E46030A8DF80030D1
:101398008DF8010004216846FFF70EFF002304E0E2
:1013A8001A1DE95CB1540133DBB2A342F8D3A11C86
:1013B800C9B2301DFFF756FFFFF794FFA11DC9B250
:1013C8003046FFF7B3FF0446FFF796FFC5462046B1
:1013D8000837BD46BDE8F081030A3B7178710421E6
:1013E8007818FFF7E9FEFFF77DFF04217818FFF76B
:1013F8009DFF0446FFF780FFE9E7000000B583B0D2
:1014080013466422009202460348006801F02BF953
:1014180003B05DF804FB00BF300000202DE9F8435D
:1014280000AF8846154602F1060902F10D0303F4E0
:10143800FC73ADEB030D6C46ADEB030D6E46030A72
:101448002370607004212046FFF7B6FEFFF74AFFBD
:101458005FFA89F221466846FFF7D0FF0446FFF796
:101468004BFF34B10DE0231DF35C08F80430013460
:10147800E4B2AC42F7D3A91CC9B2301DFFF727FF6D
:1014880004462046BD46BDE8F88310B584B0002365
:1014980002938DF80C3000938DF80430030A8DF810
:1014A80008308DF80900042102A8FFF785FEFFF730
:1014B80019FF052202A96846FFF7A0FF0446FFF7B7
:1014C8001BFF0CB99DF80440204604B010BD08B5B8
:1014D80000F0D0F908BD000038B50C4B1A780C4B59
:1014E8001978FFF723FC04460A4B40F265421A803C
:1014F800094B40F2A1121A8000F0B6F9054600F037
:10150800B3F9064B1D605860204638BD3E000020E8
:10151800000000204000002042000020340000208D
:1015280038B5FFF77BF9134C2046FFF781F9124BCA
:101538001A781044187094F8393013F0100F06D048
:101548000E4A13780133DBB21370032B0FD9094D00
:101558002846FFF7D5FD084C237818442070284604
:10156800FFF7F4FB237818442070002038BDFFF7FC
:1015780099FBECE7440000203D0000203C000020DF
:1015880030B58BB000240594069407940894099408
:10159800274B5A6942F400225A615A6902F4002220
:1015A8000192019A5A6942F480025A615A6902F416
:1015B80080020292029A5A6942F400325A615A69C8
:1015C80002F400320392039A5A6942F480225A6163
:1015D8005B6903F480230493049B164D2246402143
:1015E800284600F0A3FA4FF4005305934FF4041370
:1015F8000693079405A9104800F0BAF90C2305933F
:1016080002230693079408940723099305A94FF02A
:10161800904000F0ADF94023059301230693079409
:10162800089405A9284600F0A3F90BB030BD00BF07
:1016380000100240000400480008004872B6FEE7A7
:1016480008B50F480F4B03604FF4827343600023C3
:1016580083604FF44072C260036143614FF40072CB
:101668008261C3610362436283620722C2620363C9
:101678000823436300F083FF00B908BDFFF7DEFFCE
:10168800A40000200038004000B591B028220021B5
:1016980006A801F088F900230193029303930493A9
:1016A80005930223069301220A9210220B920D93AE
:1016B8004FF460130F9306A800F03EFA80B90F2389
:1016C800019302210291002303934FF48062049254
:1016D800059301A800F072FD20B911B05DF804FB74
:1016E800FFF7ACFFFFF7AAFF08B500F09FF8FFF778
:1016F800CBFFFFF745FFFFF7A3FF0348FFF7ECFE1B
:10170800FFF70EFFFCE700BFA400002000B583B080
:101718000C4B9A6942F001029A619A6902F001023F
:101728000092009ADA6942F08052DA61DB6903F0CC
:1017380080530193019B072000F0E4F803B05DF8A3
:1017480004FB00BF0010024000B589B000230393DA
:1017580004930593069307930268144B9A4202D0A8
:1017680009B05DF804FB03F5EC33DA6942F4804212
:10177800DA61DA6902F480420192019A5A6942F404
:1017880080225A615B6903F480230293029B4FF421
:1017980060430393022304930323069305230793CB
:1017A80003A9034800F0E4F8DAE700BF0038004076
:1017B80000040048FEE7FEE7FEE7FEE7FEE77047A5
:1017C8007047704708B500F043F808BD034AD2F8DF
:1017D800883043F47003C2F88830704700ED00E0A9
:1017E80010B504460E4B1A784FF47A73B3FBF2F334
:1017F8000C4A1068B0FBF3F000F0A6F868B90F2C9B
:1018080001D901200AE0002221464FF0FF3000F004
:101818008BF8054B1C60002000E0012010BD00BFC4
:1018280008000020040000200C00002008B5074A2A
:10183800136843F010031360032000F063F80020DE
:10184800FFF7CEFFFFF762FF002008BD002002402F
:10185800034A1168034B1B780B441360704700BFA1
:101868000801002008000020014B1868704700BFDD
:101878000801002038B50446FFF7F6FF0546B4F125
:10188800FF3F02D0044B1B781C44FFF7EDFF401BC1
:10189800A042FAD338BD00BF08000020002808DBAA
:1018A8000901C9B200F1604000F5614080F80013F9
:1018B800704700F00F000901C9B2014B1954704775
:1018C80014ED00E000B500F00700C0F1070CBCF112
:1018D800040F28BF4FF0040C031D062B0FD9C31E9D
:1018E8004FF0FF3E0EFA0CF021EA000199400EFA83
:1018F80003FE22EA0E0241EA02005DF804FB00231F
:10190800EEE70000074AD36823F4E0631B041B0CCE
:10191800000200F4E060034343F0BF6343F4003384
:10192800D360704700ED00E010B50446054BD86859
:10193800C0F30220FFF7C6FF01462046FFF7AEFFBF
:1019480010BD00BF00ED00E00138B0F1807F0BD280
:101958004FF0E0235861054AF02182F82310002057
:10196800986107221A6170470120704700ED00E076
:10197800F0B583B0002362E085685E000324B440BC
:1019880025EA0405CC68B4402C438460456825EA00
:101998000C054C68C4F300149C402C4344605FE081
:1019A800DD08083550F8254003F0070C4FEA8C0C89
:1019B8004FF00F0E0EFA0CFE24EA0E0E0C6904FA14
:1019C8000CF444EA0E0440F8254060E0032400E0EB
:1019D800002404FA0EF42C430CF1020C4F4D45F888
:1019E8002C404F4CA568D44325EA02064F6817F4EB
:1019F800801F01D042EA0506494DAE60ED6804EA51
:101A080005064F6817F4001F01D042EA0506444D49
:101A1800EE606D6804EA05064F6817F4003F01D0D0
:101A280042EA05063E4D6E602D682C404E6816F45D
:101A3800803F01D042EA0504394A146001330A683C
:101A480032FA03F468D04FF0010C0CFA03FC1CEADC
:101A58000202F3D04C6804F00304013C012C8BD93A
:101A68004C6804F00304032C0CD0C4685D004FF0EC
:101A7800030C0CFA05FC24EA0C0C8C68AC4044EA14
:101A88000C04C4604C6804F00304022C88D0046879
:101A98004FEA430E4FF0030C0CFA0EFC24EA0C0C30
:101AA8004C6804F0030404FA0EF444EA0C040460DD
:101AB8004C6814F4403FC1D01A4CA56945F00105A3
:101AC800A561A46904F001040194019C4FEA930CF8
:101AD8000CF10205114C54F8255003F0030E4FEA9F
:101AE8008E0E0F2404FA0EF425EA0405B0F1904F87
:101AF8003FF46EAF0C4CA0420AD004F58064A042BB
:101B080008D004F58064A0423FF460AF052460E784
:101B180001245EE702245CE703B0F0BD0000014049
:101B28000004014000100240000400480AB181612D
:101B38007047816270470000002800F0FF8270B58E
:101B480082B00446036813F0010F3BD0B44B5B68C6
:101B580003F00C03042B1ED0B14B5B6803F00C039D
:101B6800082B13D06368B3F5803F68D0002B40F092
:101B7800928003F1804303F504331A6822F480321B
:101B88001A601A6822F480221A605DE0A44B5B6830
:101B980013F4803FE6D04FF4003393FAA3F3A04B3D
:101BA80019684FF4003393FAA3F3B3FA83F303F0FD
:101BB8001F03012202FA03F30B4203D06368002BD0
:101BC80000F0BE82236813F0020F00F0C480944B2B
:101BD8005B6813F00C0F00F09C80914B5B6803F07E
:101BE8000C03082B00F08F802369002B00F0F08095
:101BF800012292FAA2F3B3FA83F303F1845303F5B3
:101C080084139B001A60FFF72FFE0546022393FA00
:101C1800A3F3834B1968022393FAA3F3B3FA83F36C
:101C280003F01F03012202FA03F30B4240F0C280C3
:101C3800FFF71AFE401B0228E8D9032089E2784AF8
:101C4800136843F480331360754AD36A23F00F0393
:101C5800A1680B43D3626368002B36D0FFF704FEFC
:101C680005464FF4003393FAA3F36D4B19684FF40C
:101C7800003393FAA3F3B3FA83F303F01F030122AB
:101C880002FA03F30B429DD1FFF7EEFD401B6428D7
:101C9800E7D903205DE2B3F5A02F09D0604B1A689D
:101CA80022F480321A601A6822F480221A60CBE784
:101CB80003F18043A3F53C331A6842F480221A608A
:101CC8001A6842F480321A60BEE7FFF7CDFD054678
:101CD8004FF4003393FAA3F3514B19684FF40033D0
:101CE80093FAA3F3B3FA83F303F01F03012202FA72
:101CF80003F30B423FF466AFFFF7B6FD401B6428C1
:101D0800E6D9032025E2464B5B6813F4803F7FF455
:101D18006BAF022393FAA3F3414B1968022393FA9A
:101D2800A3F3B3FA83F303F01F03012202FA03F3C8
:101D38000B4203D02369934240F004823848036879
:101D480023F0F8036169F82292FAA2F2B2FA82F259
:101D580091400B430360236813F0080F00F08C8058
:101D6800A369002B60D0012191FAA1F2B2FA82F2A4
:101D78002C4B13449B001960FFF776FD05460223A0
:101D880093FAA3F293FAA3F293FAA3F2244A516ABC
:101D980093FAA3F3B3FA83F303F01F03012202FAC1
:101DA80003F30B4268D1FFF75FFD401B0228E6D919
:101DB8000320CEE11A48036823F0F8036169F8228A
:101DC80092FAA2F2B2FA82F291400B430360C2E7A0
:101DD800012393FAA3F3B3FA83F303F1845303F5CE
:101DE80084139B0000221A60FFF73EFD054602237C
:101DF80093FAA3F30A4B1968022393FAA3F3B3FAED
:101E080083F303F01F03012202FA03F30B42A2D06B
:101E1800FFF72AFD401B0228E9D9032099E100BFFA
:101E28000010024020819010012292FAA2F2B2FA28
:101E380082F2B74B13449B0000221A60FFF714FD8F
:101E48000546022393FAA3F293FAA3F293FAA3F2B4
:101E5800B04A516A93FAA3F3B3FA83F303F01F036A
:101E6800012202FA03F30B4206D0FFF7FDFC401BE8
:101E78000228E6D903206CE1236813F0040F00F070
:101E8800A980A44BDB6913F0805F20D1A14BDA69EC
:101E980042F08052DA61DB6903F080530193019BC1
:101EA80001259D4B1B6813F4807F12D0E368012B3A
:101EB80023D073BB03F1804303F504331A6A22F07D
:101EC80001021A621A6A22F004021A621AE0002554
:101ED800E7E7914A136843F480731360FFF7C4FC83
:101EE80006468D4B1B6813F4807FDFD1FFF7BCFCDF
:101EF800801B6428F5D903202BE1864A136A43F036
:101F080001031362E368002B3CD0FFF7ADFC0646E3
:101F18002EE0052B09D07F4B1A6A22F001021A62C3
:101F28001A6A22F004021A62ECE77A4B1A6A42F043
:101F380004021A621A6A42F001021A62E2E70223F4
:101F480093FAA3F3734B596A022393FAA3F3B3FAF0
:101F580083F303F01F03012202FA03F3194238D175
:101F6800FFF782FC801B41F28833984200F2EC8034
:101F7800022393FAA3F293FAA3F3002BDFD0654B65
:101F8800196AE1E7FFF770FC064618E0022393FAA6
:101F9800A3F3604B596A022393FAA3F3B3FA83F3CA
:101FA80003F01F03012202FA03F3194211D0FFF7CD
:101FB8005BFC801B41F28833984200F2C780022301
:101FC80093FAA3F293FAA3F3002BDFD0514B196ACB
:101FD800E1E7B5BBE369002B00F0BA804D4A5268CF
:101FE80002F00C02082A00F09980022B2FD04FF043
:101FF800807393FAA3F3B3FA83F303F1845303F5DD
:1020080084139B0000221A60FFF72EFC04464FF051
:10201800007393FAA3F33F4B19684FF0007393FAD8
:10202800A3F3B3FA83F303F01F03012202FA03F3C5
:1020380019426BD0FFF718FC001B0228E7D90320D0
:1020480087E0344AD36923F08053D361C2E74FF065
:10205800807393FAA3F3B3FA83F303F1845303F57C
:1020680084139B0000221A60FFF7FEFB05464FF021
:10207800007393FAA3F3274B19684FF0007393FA90
:10208800A3F3B3FA83F303F01F03012202FA03F365
:10209800194206D0FFF7E8FB401B0228E7D90320C6
:1020A80057E01C494B6823F47413626A206A0243A0
:1020B80013434B604FF0807393FAA3F3B3FA83F39F
:1020C80003F1845303F584139B0001221A60FFF780
:1020D800CBFB04464FF0007393FAA3F30D4B19683A
:1020E8004FF0007393FAA3F3B3FA83F303F01F03DB
:1020F800012202FA03F3194206D1FFF7B5FB001BD0
:102108000228E7D9032024E0002022E0002020E074
:10211800208190100010024000700040012B1AD05E
:10212800104B5B6803F48031226A914215D103F4A5
:102138007013626A934212D100200AE001207047AE
:10214800012006E0012004E0032002E0032000E073
:10215800002002B070BD0120FBE70120F9E7012053
:10216800F7E700BF001002400F4B5B6803F00C025A
:10217800082A01D00D487047C3F383420C49885C94
:10218800094AD26A02F00F020A498A5C13F4803FB6
:1021980005D0064BB3FBF2F303FB00F07047064B88
:1021A80003FB00F0704700BF0010024000127A00E5
:1021B800482A0008382A000800093D00002800F0D5
:1021C800BE8070B50D460446614B1B6803F00703DB
:1021D8008B420BD25E4A136823F007030B4313604C
:1021E800136803F007038B4240F0AB80236813F0B9
:1021F800020F06D0574A536823F0F003A1680B4337
:102208005360236813F0010F5AD06368012B2DD057
:10221800022B40D0022292FAA2F24E4A1068022201
:1022280092FAA2F2B2FA82F202F01F02012101FA36
:1022380002F2104200F0878046494A6822F0030201
:1022480013434B60FFF710FB0646424B5B6803F0F5
:102258000C036268B3EB820F32D0FFF705FB801BDB
:1022680041F288339842F0D9032067E04FF40032F6
:1022780092FAA2F2374A10684FF4003292FAA2F2A8
:10228800B2FA82F202F01F02012101FA02F20242BE
:10229800D2D1012052E04FF0007292FAA2F22D4AF8
:1022A80010684FF0007292FAA2F2B2FA82F202F0CB
:1022B8001F02012101FA02F21042BDD101203DE0C6
:1022C800234B1B6803F00703AB420AD9204A136863
:1022D80023F007032B431360136803F00703AB4293
:1022E80033D1236813F0040F06D01A4A536823F435
:1022F800E063E1680B435360236813F0080F07D0CD
:10230800144A536823F46053216943EAC1035360B4
:10231800FFF72AFF0F4B5B6803F0F003F02292FAF5
:10232800A2F2B2FA82F2D3400B4AD35CD8400B4BEC
:1023380018600B4B1868FFF753FA002070BD012096
:1023480070470120FAE70120F8E70120F6E700BF0F
:102358000020024000100240282A00080400002043
:102368000C0000202DE9F04782B005468846174644
:102378001E46FFF779FA0A9B1B1A03EB0609FFF7BB
:1023880073FA8246284B1B68C3F3CB3309FB03F36C
:1023980001932B689C6838EA04040CBF01230023CE
:1023A800BB423DD0B6F1FF3FF3D0FFF75DFAA0EB9B
:1023B8000A00484507D2019A02B14A46019B013BEF
:1023C80001939146E5E72A68536823F0E0035360D8
:1023D8006B68B3F5827F0BD0AB6AB3F5005F14D09E
:1023E800012385F85D30002385F85C30032018E070
:1023F800AB68B3F5004F02D0B3F5806FECD12A6813
:10240800136823F040031360E6E72A68136823F48F
:10241800005313602A68136843F400531360DFE71E
:10242800002002B0BDE8F087040000202DE9F04745
:1024380082B006460C4615461F4600238DF8033029
:10244800FFF712FA0A9B1B1A03EB0708FFF70CFAAF
:102458008146D6F800A0304B1B6803EB8303C3EB1F
:10246800C3031B0D08FB03F3019302E0B7F1FF3F21
:1024780012D133689B6803EA040CAC4547D0B4F525
:10248800C06FF3D1002DF1D19AF80C30DBB28DF882
:1024980003309DF80330E9E7FFF7E6F9A0EB090000
:1024A800404507D2019A02B14246019B013B019384
:1024B8009046DEE73268536823F0E00353607368A0
:1024C800B3F5827F0BD0B36AB3F5005F14D0012354
:1024D80086F85D30002386F85C30032018E0B36886
:1024E800B3F5004F02D0B3F5806FECD132681368B2
:1024F80023F040031360E6E73268136823F40053BF
:1025080013603268136843F400531360DFE7002058
:1025180002B0BDE8F08700BF0400002070B582B0AB
:1025280004460D46164600920B4600224FF4C05151
:10253800FFF77CFFB0B900962B4600228021204689
:10254800FFF710FFA8B900962B4600224FF4C06190
:102558002046FFF76BFF50B1236E43F0200323663C
:10256800032004E0236E43F020032366032002B017
:1025780070BD236E43F0200323660320F7E700288D
:102588006FD010B50446436A33B94368B3F5827F08
:1025980005D00023C36102E00023036143610023E7
:1025A800A36294F85D30002B52D0022384F85D308A
:1025B8002268136823F040031360E368B3F5E06F03
:1025C8004CD90022B3F5706F04D0B3F5E06F01D099
:1025D8000023A362636803F48273A16801F40441D1
:1025E8000B43216901F002010B43616901F001010C
:1025F8000B43A16901F400710B43E16901F0380153
:102608000B43216A01F080010B43A16A01F40051D8
:1026180020680B430360638B03F00403616A01F0D5
:1026280010010B43616B01F008010B43E16801F4F1
:1026380070610B43216813434B602268D36923F40C
:102648000063D36100202066012384F85D3010BD4B
:1026580084F85C302046FFF777F8A6E74FF48052FD
:10266800B0E7012070472DE9F8431F46089D90F810
:102678005C30012B00F06B810446884691460123AB
:1026880080F85C30FFF7F0F8064694F85D30DBB26E
:102698006268012B0AD0B2F5827F40F04681A268B9
:1026A800002A40F04881042B40F04781B8F1000F20
:1026B80000F04581B9F1000F00F04381002F00F0D0
:1026C800428194F85D30DBB2042B02D0052384F8F4
:1026D8005D3000232366C4F84090A4F84670A4F83F
:1026E8004470C4F83880E787A787E3642365E36804
:1026F800B3F5E06F01D8012F23D92268536823F47A
:102708008053536023681A6812F0400F03D11A6887
:1027180042F040021A60E368B3F5E06F5CD9636881
:102728000BB1012F0BD1A26B23681288DA60A36B5F
:102738000233A363E38F9BB2013B9BB2E38701277C
:1027480030E02268536843F480535360DAE7A26BA1
:102758001288DA60A36B0233A363E38F9BB2013B59
:102768009BB2E387002723689A6812F0010F11D003
:10277800B4F8462092B26AB1DA68236C1A80236CE6
:1027880002332364B4F846309BB2013B9BB2A4F8F1
:1027980046300127FFF768F8831BAB4202D3B5F137
:1027A800FF3F14D1E38F9BB22BB9B4F846309BB2EC
:1027B800002B00F0AB8023689A6812F0020FD2D089
:1027C800E28F92B2002ACED0002FCCD0BFE70123EF
:1027D80084F85D300320A9E063680BB1012F0FD1A5
:1027E800E38F9BB2012B0DD9A26B23681288DA60A4
:1027F800A36B0233A363E38F9BB2023B9BB2E387D5
:10280800012749E0A26B236812781A73A36B01337E
:10281800A363E38F9BB2013B9BB2E387F0E7E28FB0
:1028280092B2012A0CD9A26B1288DA60A36B023328
:10283800A363E38F9BB2023B9BB2E38700273DE093
:10284800A26B12781A73A36B0133A363E38F9BB255
:10285800013B9BB2E387002730E02268536843F4CA
:102868008053536001270DE0226C1B7B1370236C8F
:1028780001332364B4F846309BB2013B9BB2A4F801
:1028880046300127FEF7F0FF801BA84202D3B5F1BE
:10289800FF3F36D1002D34D0E38F9BB223B9B4F873
:1028A80046309BB2002B31D023689A6812F0020F91
:1028B80004D0E28F92B20AB1002FB0D123689A688F
:1028C80012F0010FDED0B4F8462092B2002AD9D017
:1028D800B4F8462092B2012AC6D9DA68236C1A8065
:1028E800236C02332364B4F846309BB2023B9BB29C
:1028F800A4F84630B4F846309BB2012BADD9012775
:10290800C0E7012384F85D3003200FE032462946F2
:102918002046FFF703FE10B1202323660120236E13
:102928009BB9012384F85D3000E00220002384F87D
:102938005C30BDE8F8830220F8E70220F6E70120C2
:10294800F4E70120F2E70120F0E70120EEE702209A
:10295800EFE70000DFF834D0FEF738FF0C480D49E8
:102968000D4A002302E0D458C4500433C4188C42E2
:10297800F9D30A4A0A4C002301E013600432A24248
:10298800FBD300F019F8FEF7AFFEFEE70040002089
:102998000000002010000020602A0008100000201D
:1029A8000C010020FEE702440346934200D1704721
:1029B80003F8011BF9E7000070B50D4D0D4C641BC1
:1029C800A4100026A64209D10B4D0C4C00F018F8B3
:1029D800641BA4100026A64205D170BD55F8043B1F
:1029E80098470136EEE755F8043B98470136F2E779
:1029F800582A0008582A0008582A00085C2A0008A3
:102A0800F8B500BFF8BC08BC9E467047F8B500BFD3
:082A1800F8BC08BC9E467047A3
:102A2000FFFFFFFFFFFF00000000000000000000AC
:102A3000010203040607080901020304050607084A
:102A4000090A0B0C0D0E0F100203040506070809F6
:082A50000A0B0C0D0E0F101013
:042A58000908000861
:042A5C00E507000882
:102A60000F00000000127A000100000010000000BA
:040000050800295D69
:00000001FF
